:100000000C947F010C94EE130C949C010C949E01B3
:100010000C949C010C949C010C949C010C949C01EC
:100020000C949C010C949C010C949C010C949C01DC
:100030000C949C010C949C010C949C010C949C01CC
:100040000C949C010C949C010C949C010C949C01BC
:100050000C949C010C949C010C949C010C949C01AC
:100060000C949C010C949C011201100100000008EA
:10007000828201320104010200011201100100001C
:100080000008828201330104010200010501090414
:10009000A10185010901A100093009311580257FE1
:1000A000750895028102093309341580257F75088A
:1000B000950281020939150025077505950181030F
:1000C0007503950181030509190129101500250102
:1000D00075019510550065008102C0C00501090435
:1000E000A10185010901A100093009311580257F91
:1000F000750895028102093309341580257F75083A
:1001000095028102093915002507750595018103BE
:1001100075039501810305091901291015002501B1
:1001200075019510550065008102C0C005010904E4
:10013000A10185020901A100093009311580257F3F
:10014000750895028102093309341580257F7508E9
:10015000950281020939150025077505950181036E
:100160007503950181030509190129101500250161
:1001700075019510550065008102C0C00501090296
:10018000A10185010901A100050919012903150033
:10019000250195047501810295017504810305010E
:1001A0000930093109381580257F750895038106C6
:1001B000C0C00904A10185020901A100093009316B
:1001C0001580257F750895028102C005091901294E
:1001D000101500250175019510550065008102C0BC
:1001E00005010904A10185010901A10009300931B6
:1001F0001580257F750895028102093915002507AC
:1002000075059501810375039501810305091901A0
:100210002910150025017501951055006500810212
:100220000501093609360936150026FF00750895BF
:10023000038102C0C005010904A10185010901A1D2
:1002400000093009311580257F7508950281020962
:100250003309341580257F75089502810209391507
:100260000025077505950181037503950181030537
:100270000919012910150025017501951055006512
:1002800000810205010936093609360936093609A1
:100290003609360936093609360936093615002673
:1002A000FF00750895018102C0C0FF0004FF06072A
:1002B00005FF020103FFFFFFFFFFFF0206FF04032C
:1002C00005FF000107FFFFFF00020104FF03FF0617
:1002D00007FFFF05040309040A034D006F004A00ED
:1002E0006F001C0352006500740072006F00200054
:1002F0004100640061007000740065007200112408
:100300001FBECFEFD4E0DEBFCDBF11E0A0E0B1E073
:10031000ECE8FAE202C005900D92A432B107D9F7D9
:1003200011E0A4E2B1E001C01D92AE3CB107E1F7DB
:100330000E94B5050C9444150C94000078946F93BA
:100340006FB72F933F934F935F9353B15C73452FD8
:10035000447130918D01347120918C01403049F00D
:10036000403161F0443179F03030A1F0343181F026
:1003700012C0303179F0343059F00DC0343151F0C1
:10038000303031F008C0343029F0303109F003C08A
:10039000239501C02A9520938C01452F48723091F6
:1003A0008D01387220918B01403049F0403261F06C
:1003B000483279F03030A1F0383281F012C030325A
:1003C00079F0383059F00DC0383251F0303031F01A
:1003D00008C0383029F0303209F003C0239501C03D
:1003E0002A9520938B0150938D015F914F913F91FE
:1003F0002F916FBF6F9118950F931F93FF93EF93FA
:10040000BF93AF93F92FE82F09E000938F0100E22B
:100410000093900100E00093910101E000939201AC
:1004200001E00093930100E0009394010093950193
:100430000093960109E20093970107D0BF91AF9115
:10044000EF91FF911F910F910895A1E0BFE809E09E
:100450002D980000000000002C9800000000000013
:100460002C9A000000002C980000000000002C9A3C
:100470000000000000002C980000000000002C9AF2
:100480000000000000002C980000000000002C9AE2
:1004900000000000000000002D9A1D9117FD2C9A0D
:1004A00017FF2C982D98000000002C9A16FD2D9A0D
:1004B00016FF2D982C9A000000002D9A15FD2C9AFD
:1004C00015FF2C982D9A000000002C9A14FD2D9AEF
:1004D00014FF2D982C9A000000002D9A15FD2C9ADF
:1004E00015FF2C982D9A000000002C9A14FD2D9ACF
:1004F00014FF2D982C9A000000002D9A15FD2C9ABF
:1005000015FF2C982D9A000000002C9A14FD2D9AAE
:1005100014FF2D982C9A000000002D9A0A952D9A10
:100520002C9A0895F92FE82F21E030E0E20FF31F15
:100530002227332744275527662777278827992797
:1005400090E099D0B6D082D0292F80D0392F7ED09C
:10055000492F253021F0293089F180E00895BFEF3F
:10056000BA95F1F7B8ECBA95F1F791E084D0A1D043
:100570006DD0292F6BD0392F69D0492F67D0592FD3
:1005800040835195518340E050E027FD416026FDB6
:10059000426025FD526024FD51602F7035FD40649E
:1005A00034FD406833FD446032FD486031FD4061F8
:1005B00030FD406245835683822F0895B4E6BA9594
:1005C000F1F790E458D093E056D092E054D071D037
:1005D0003DD0292F3BD0392F39D0492F37D0592F33
:1005E00035D0692F33D0792F31D0892F2FD0405873
:1005F000505851954083518360586195705871955A
:100600006283738340E050E020FD416021FD426041
:1006100022FD486023FD406124FD516034FD52609D
:1006200035FD406836FD4064803408F04064903405
:1006300008F04068458356833F70232F3E7F31FD8D
:1006400031603D7F20FD3260832F089590E0B4E15A
:10065000A8E0BA9579F01899FCCFB9E0BA95F1F70E
:10066000990F18999160B4E1BA9521F0189BFCCFCD
:10067000AA9579F70895A8E097FD0DC0209ABDE0EE
:10068000BA95F1F700002098B3E0BA95F1F7990F09
:10069000AA9591F70895209AB3E0BA95F1F7000072
:1006A00000002098BDE0BA95F1F7990FAA9521F7BF
:1006B0000895209AB3E0BA95F1F700000000209861
:1006C00008951AB889EF8BB914B88FE385B917B8B4
:1006D00088B9089580918601823009F459C0833029
:1006E00030F4882359F0813009F0C0C02CC0833029
:1006F00009F473C0843009F0B9C094C088E690E072
:10070000909325018093240182E190E0909327014A
:10071000809326018CE890E0909388018093870174
:1007200080E590E090938A018093890181E0809335
:10073000810188E291E0909384018093830188E0B5
:100740008093850193C088E690E090932501809383
:10075000240182E190E090932701809326018CEDA3
:1007600090E0909388018093870180EA90E09093D5
:100770008A018093890182E08093810188E291E07F
:10078000909384018093830188E0809385016EC0FB
:100790008AE790E0909325018093240182E190E024
:1007A00090932701809326018CE791E09093880134
:1007B0008093870184E690E090938A018093890179
:1007C00082E08093810180E391E0909384018093A3
:1007D000830185E08093850149C088E690E090938D
:1007E00025018093240182E190E09093270180937A
:1007F000260180EE91E0909388018093870185E542
:1008000090E090938A018093890181E08093810137
:1008100085E391E0909384018093830189E0809344
:10082000850124C088E690E09093250180932401FF
:1008300082E190E0909327018093260185E392E086
:10084000909388018093870185E790E090938A01D7
:100850008093890181E0809381018EE391E0909300
:1008600084018093830184E18093850180918901D3
:1008700080931901F894EAE2F0E08081826080833D
:1008800080818660808326EF39E047E751E0CA0126
:100890000197F1F721503040D1F7EAE2F0E0808192
:1008A0008D7F80838081897F808378940895FC0187
:1008B000808180768032F9F48181813059F4809191
:1008C0008301909184019093B3018093B201809150
:1008D00085010895823041F482E891E09093B3015C
:1008E0008093B20181E008958A3029F48381809356
:1008F000820180E0089580E00895FC0181818630C6
:1009000031F58381823081F0823219F08130F9F43F
:1009100013C080918701909188019093B3018093D7
:10092000B20180918901089580E091E09093B30134
:100930008093B20182E20895809124019091250173
:100940009093B3018093B20180912601089580E0D5
:1009500008950F931F93082FA8E2B1E0E2E5F1E0BC
:1009600088E001900D928150E1F78FEF80932D0187
:1009700000932801A0E3B1E0EAE5F1E085E0019011
:100980000D928150E1F700933001A5E3B1E0EFE56E
:10099000F1E089E001900D928150E1F78FEF8093B3
:1009A000380100933501AEE3B1E0E8E6F1E084E11F
:1009B00001900D928150E1F78FEF809343010093F6
:1009C0003E0110928601359981C034996AC086B182
:1009D00090E08E7190708630910531F187309105ED
:1009E0004CF482309105B1F08430910519F1892BD6
:1009F00059F008C08A30910579F18C30910501F1E8
:100A0000089781F190E072C088E291E00E94261080
:100A100010E086C088E291E065E371E04EE351E0CA
:100A20000E94EC0E10E07CC088E291E00E944B092D
:100A300010E076C088E291E00E94170A10E05BC0E7
:100A400082E080938601013009F08AC080E391E062
:100A50000E940D0611E064C088E291E00E94E20865
:100A600010E05EC083B190E0867090708230910596
:100A700091F08630910519F0892B39F036C088E263
:100A800091E00E94510810E04BC088E291E00E9482
:100A9000E80710E045C088E291E00E94420A10E0B9
:100AA0003FC0339906C088E291E00E94D91110E05E
:100AB00037C0023011F090E005C088E291E00E945A
:100AC0000D0D91E081E08093860110C0339907C03D
:100AD00088E291E0602F0E947D0610E021C088E24C
:100AE00091E00E94530B10E006C091E0992311F0B1
:100AF00010E016C010E089B1897071F44C9B05C0FC
:100B000088E291E00E9448060BC088E291E060E331
:100B100071E00E94790D04C088E291E00E948F0A82
:100B20000230B1F480918601823091F441E351E0CA
:100B300029E231E0D9018D91FA0181938C91808372
:100B4000F9018581FA018283F9018681FA018383A3
:100B5000112341F4E8E6F0E080818E7F808302C0BB
:100B600011E0C9CF1F910F910895CF92DF92EF92BC
:100B7000FF920F931F93CF93DF930E9461030E9414
:100B80005D121092860181E00E94A9040E946A030E
:100B9000FF24F394EE24EA94C3EAD1E0CC24C39476
:100BA000DD240E946F12888184FFFBCF8F2D0E946D
:100BB000A90400918501093078F41D2D03C0185F48
:100BC000093058F48091830190918401810F911D27
:100BD000602F0E94AB1312C01D2D80918301909154
:100BE0008401810F911D68E00E94AB1308500E94A0
:100BF0006F12888184FFFBCF002309F7F394809163
:100C000081018F1508F4FC2C80918601E81649F2C9
:100C10000E946A03E0908601C4CFDC01E4E2F0E0C8
:100C20008081817C8083E5E2F0E080818E63808337
:100C3000E7E2F0E080818E7F8083E8E2F0E080816F
:100C4000816080838CE380936B0081E080936800F7
:100C500080918C0112968C93129780918B01139640
:100C60008C93139710928C0110928B01199907C0E5
:100C700011968C911197816011968C9311973099F0
:100C800006C011968C911197826011968C930895ED
:100C90000F931F938C01E5E2F0E080818E7F8083CB
:100CA000E4E2F0E080818E7F8083EBE2F0E08081FF
:100CB0008F778083EAE2F0E0808180688083C801DA
:100CC0000E949202EAEBF2E0E80FF11DE491D801F4
:100CD0001596EC931F910F910895E4E2F0E02081C6
:100CE000277F2083208120632083E5E2F0E02081BC
:100CF000286320830E94FC010895DC01EAE2F0E011
:100D000080818E7E8083EBE2F0E080818161808350
:100D1000E4E2F0E080818863808380818D7F80833E
:100D2000E5E2F0E0808182608083E7E2F0E08081AC
:100D3000807E8083E8E2F0E080818F618083489B41
:100D40000BC0E4E2F0E0808184608083E5E2F0E0C3
:100D50008081837C808314C0E4E2F0E080818B7F1B
:100D60008083E5E2F0E080818C638083E7E2F0E05D
:100D700080818E7F8083E8E2F0E0808181608083E3
:100D800087E180937E00EAE7F0E085E0808384E6F7
:100D900080937C00808180688083808186FDFDCF88
:100DA000613009F5EAE7F0E080818064808380812A
:100DB00086FDFDCF909179008FE7891B12968C9369
:100DC000129782E680937C00EAE7F0E080818064FD
:100DD0008083808186FDFDCF909179008FE7891B0C
:100DE00011968C931197489B29C081E080938601CE
:100DF000623021F581E680937C00EAE7F0E08081B3
:100E000080648083808186FDFDCF909179008FE79B
:100E1000891B11968C93119780E680937C00EAE7FA
:100E2000F0E0808180648083808186FDFDCF909199
:100E300079008FE7891B12968C93129710927A0093
:100E400010927E00489B17C04C9909C0613039F45C
:100E500016968C911697816016968C931697199911
:100E60009AC0623009F097C016968C9116978160EF
:100E700016968C93089510928601E5E2F0E0808149
:100E8000877F808385E08A95F1F7309907C01696B1
:100E90008C911697826016968C9316971A9907C0B4
:100EA00016968C911697806116968C9316971999C1
:100EB00007C016968C911697806816968C93169795
:100EC0004C9907C017968C911797846017968C934E
:100ED0001797E5E2F0E080818860808380818F7ED3
:100EE000808385E08A95F1F7309907C016968C913A
:100EF0001697846016968C9316971A9907C01696C3
:100F00008C911697806216968C931697199907C044
:100F100017968C911797816017968C9317974C9919
:100F200007C016968C911697816016968C9316972B
:100F3000E5E2F0E080818061808380818F7D808325
:100F400085E08A95F1F7309907C016968C9116972F
:100F5000886016968C9316971A9907C016968C91EE
:100F60001697806416968C931697199907C0179652
:100F70008C911797826017968C9317974C9906C09F
:100F800017968C911797886017968C93E5E2F0E09E
:100F9000808180628083089590E020E0A3E2B0E049
:100FA000EBE2F0E034E1220F8C9180FD2160808142
:100FB0008F778083832F8A95F1F780818068808383
:100FC000832F8A95F1F79F5F983069F7822F0895F4
:100FD000CF93DF93EC01ABE2B0E08C91886F8C9300
:100FE0008C918E7F8C93EAE2F0E08081896C808323
:100FF00080818F7C8083E4E2F0E080818E7F80833B
:10100000E5E2F0E08081816080838C918F7B8C931E
:101010000E94CC07282F30E0C901807F9070803477
:101020009105E1F520FF02C080E8898321FF02C01D
:101030008FE7898322FF02C080E88A8323FF02C0F2
:101040008FE78A830E94CC07282F982F81FF03C047
:101050008E8180648E8392FF03C08E8180688E8330
:1010600093FF03C08F8182608F8394FF03C08F81C1
:1010700081608F8395FF03C08E8184608E8396FF8D
:1010800003C08E8182608E8322231CF48E81816056
:101090008E83EBE2F0E0808180648083DF91CF91EA
:1010A0000895DC01EAE2F0E0808186708083EBE263
:1010B000F0E08081896F8083E4E2F0E08081807CD1
:1010C0008083E5E2F0E080818F638083E9E2F0E0F5
:1010D0008081982F9170808183FD926080917D0145
:1010E000981709F44BC09130A9F0913028F0923054
:1010F00069F19330C1F51CC0813029F48FE7119656
:101100008C93119730C0823071F580E811968C93E2
:10111000119729C0833029F48FE711968C9311978A
:1011200022C0882301F580E811968C9311971BC08B
:10113000823029F48FE711968C93119714C0813077
:1011400091F480E811968C9311970DC0882329F4AF
:101150008FE711968C93119706C0833021F480E8B5
:1011600011968C93119790937D0183E080937C017D
:1011700011968C91119780937E010CC080917C0117
:10118000882341F0815080937C0180917E011196EB
:101190008C9311974E9906C016968C911697816084
:1011A00016968C930895EBE2F0E080818F7E808329
:1011B00089E191E00197F1F789B190819061908385
:1011C00081700895CF93DF93EC01E4E2F0E0808139
:1011D000837C8083808182608083A5E2B0E08C91F3
:1011E0008E638C93EAE2F0E080818E7F8083808141
:1011F00080618083EBE2F0E08081816180838C916B
:101200008D7F8C931D9902C080E88A831C9902C04F
:101210008FE78A831B9902C080E889831A9902C0EC
:101220008FE789830E94D308882319F48E81826016
:101230008E830E94D308882319F48E8181608E8367
:101240000E94D308882319F48E8188608E830E94BF
:10125000D308882319F48E8184608E830E94D3087A
:10126000882319F48E8180688E830E94D308882396
:1012700019F48E8180648E830E94D308882319F428
:101280008F8181608F83E5E2F0E0808182608083DE
:10129000DF91CF910895CF93DF93DC01E4E2F0E09A
:1012A0008081837C8083808182608083E5E2F0E0BE
:1012B00080818E638083EAE2F0E0808180618083B8
:1012C000EBE2F0E080818F7E808392E02BE230E0E1
:1012D000E3E2F0E065E270E040E85FE7E901888181
:1012E0008F7E88830000000080818C7309F447C0E2
:1012F000808185FD03C012964C931297808184FDF6
:1013000003C011965C931197808183FD03C01296F0
:101310005C931297808182FD03C011964C931197C4
:10132000EB0188818D7F888300000000808185FD2E
:1013300007C016968C911697816016968C93169717
:10134000808184FD07C016968C9116978260169650
:101350008C931697808183FD07C017968C91179701
:10136000826017968C931797808182FD36C01796FE
:101370008C911797816017968C9317972EC0EB016D
:1013800088818D7F888300000000808185FD07C0F3
:1013900016968C911697846016968C93169780817A
:1013A00084FD07C016968C911697886016968C93CC
:1013B0001697808183FD07C016968C9116978061E1
:1013C00016968C931697808182FD07C016968C9195
:1013D0001697806216968C931697E9018881806132
:1013E0008883EB01888182608883915009F076CFF1
:1013F000DF91CF91089590E020E0E5E2F0E034E65F
:10140000A3E2B0E080818B7F8083832F8A95F1F700
:1014100026958C9185FD2068808184608083832F50
:101420008A95F1F79F5F983069F7822F0895EF92C0
:10143000FF920F931F937C0105E210E0F801808179
:101440008C7E8083808184628083E4E2F0E080810E
:101450008F7D808380818C618083F80180818860AA
:1014600080838AEF8A95F1F70E94FB09F801808159
:10147000877F80838AEAF70187831F910F91FF900E
:10148000EF900895DC01EAE2F0E0808186708083CD
:10149000EBE2F0E08081896F8083E4E2F0E080811C
:1014A0008E7F8083E5E2F0E08081816080834E99C9
:1014B0000CC016968C911697816016968C93169791
:1014C00004C09F5F9B3F21F4089590E0E3E2F0E0C9
:1014D000808180FDF6CF89B1982F892F8095282FA4
:1014E000217093FF226094FF246095FF286090E0B4
:1014F000E3E2F0E003C09F5F9B3F81F0808180FFCB
:10150000FACF89B180FF206183FF206284FF2064CD
:1015100085FF20688FE7821B11968C930895DC016C
:10152000EAE2F0E080818678808380818068808331
:10153000EBE2F0E080818F77808380818967808310
:10154000E4E2F0E080818E7F8083E5E2F0E080815C
:101550008160808386E48A95F1F789B1807311F008
:1015600090E015C04E9907C016968C911697816031
:1015700016968C931697189B02C091E008C0179698
:101580008C911797816017968C93179791E0EBE2F7
:10159000F0E080818068808386E48A95F1F748993D
:1015A00004C080E812968C9312974B9904C08FE781
:1015B00012968C9312974C9904C080E811968C93E4
:1015C00011974D9904C08FE711968C931197992329
:1015D00091F44E9907C016968C91169781601696D5
:1015E0008C931697189959C016968C91169782600D
:1015F00016968C9352C04E9907C016968C911697EA
:10160000826016968C931697189907C016968C913F
:101610001697846016968C931697EBE2F0E0808123
:101620008F77808396E4892F8A95F1F7808180688F
:101630008083892F8A95F1F780818F7780839A95AF
:10164000F1F789B1897349F580818068808386E4E8
:101650008A95F1F7489907C016968C911697806283
:1016600016968C9316974B9907C016968C911697E1
:10167000806116968C9316974C9907C016968C919C
:101680001697886016968C9316974D9906C01796F4
:101690008C911797846017968C93EBE2F0E0808131
:1016A000806880830895DC01E4E2F0E08081817C41
:1016B0008083E5E2F0E080818E638083E7E2F0E002
:1016C0008081807C8083E8E2F0E080818F6380838A
:1016D000EAE2F0E080818E7E8083EBE2F0E08081C0
:1016E000816180831D9907C016968C91169780643E
:1016F00016968C9316971C9907C016968C91169780
:10170000886016968C9316971B9907C016968C9135
:101710001697806216968C9316971A9907C017969B
:101720008C911797816017968C931797199907C01A
:1017300017968C911797826017968C93179732990A
:1017400007C016968C911697806816968C931697FC
:10175000319907C016968C911697846016968C93D3
:101760001697309906C016968C911697806116963A
:101770008C930895DC0186E48A95F1F783B18C702F
:1017800011F090E015C0199907C016968C91169724
:10179000816016968C931697319B02C091E008C029
:1017A00016968C911697806416968C93169791E0F6
:1017B000E8E2F0E080818460808386E48A95F1F736
:1017C0001D9904C080E812968C9312971C9904C04E
:1017D0008FE712968C9312971B9904C080E811969C
:1017E0008C9311971A9904C08FE711968C931197D7
:1017F000992391F4199907C016968C9116978160D8
:1018000016968C931697319959C016968C91169707
:10181000826016968C930895199907C016968C913C
:101820001697826016968C931697319907C0169674
:101830008C911697846016968C931697E8E2F0E0E8
:1018400080818B7F808396E4892F8A95F1F7808150
:1018500084608083892F8A95F1F780818B7F8083D4
:101860009A95F1F783B18C7349F580818460808308
:1018700086E48A95F1F71D9907C016968C91169704
:10188000806216968C9316971C9907C016968C91B9
:101890001697806116968C9316971B9907C016961B
:1018A0008C911697886016968C9316971A9906C095
:1018B00016968C911697806416968C93089583B132
:1018C000E8E2F0E090819D7F908328E7922F9A953F
:1018D000F1F79081926090832A95F1F7869586952D
:1018E000809581700895CF93DF93EC01E4E2F0E0FE
:1018F00080818B7F8083E5E2F0E08081846080835B
:10190000E7E2F0E0808184608083A8E2B0E08C911F
:1019100084608C938081826080838C9182608C93C0
:1019200080EF8A95F1F78C918B7F8C9388E78A956D
:10193000F1F70E945F0C882319F08E8181608E83FD
:101940000E945F0C882319F08E8182608E830E9432
:101950005F0C882319F08F8182608F830E945F0C57
:10196000882319F08F8181608F830E945F0C882308
:1019700011F080E88A830E945F0C882311F08FE7C2
:101980008A830E945F0C882311F080E889830E947B
:101990005F0C882311F08FE789830E945F0C8823F6
:1019A00019F08E8188608E830E945F0C882319F065
:1019B0008E8180618E830E945F0C882319F08E8156
:1019C00084608E830E945F0C882319F08E81806270
:1019D0008E830E945F0C882321F08E81837C8E830E
:1019E00019C08E81282F247E2E83982F80FF03C05C
:1019F000822F82608E8391FF03C08E8180618E83EF
:101A000093FF03C08E8181608E8394FF03C08E811B
:101A100088608E83DF91CF9108959C01E4E2F0E02D
:101A20008081817C8083E5E2F0E080818E63808329
:101A3000E7E2F0E080818460808380818D7F808315
:101A4000E8E2F0E080818260808380818B7F808308
:101A500083B1887321F4C9010E94730C0895C901F0
:101A60000E94BA0B0895282F269511F437E009C07B
:101A700037E0982F990F822F8170892B315026954E
:101A8000C1F790E002C0880F991F3A95E2F70895D8
:101A900089B1E5E2F0E090819E7F908328E7922F64
:101AA0009A95F1F79081916090832A95F1F782954C
:101AB0008695877080958170089520E090E0A9E276
:101AC000B0E0E5E2F0E038E726958C9185FF2068EC
:101AD00080818E7F8083832F8A95F1F7808181605A
:101AE0008083832F8A95F1F79F5F983069F7822F63
:101AF0000895AF92BF92DF92EF92FF920F931F93E0
:101B0000CF93DF93EC015B01EAE2F0E080818F7D0F
:101B10008083ABE2B0E08C9180628C93808180689E
:101B200080838C9180688C93E4E2F0E08081816016
:101B30008083E5E2F0E080818160808380EF8A9598
:101B4000F1F78C918F778C9388E78A95F1F70E9453
:101B50005D0DF82E0E945D0DD82E0E945D0D482F60
:101B6000FF2014F48FE789832F2D30E0F6FE02C0AA
:101B700080E8898325FF02C08FE78A8324FF02C0A3
:101B800080E88A83D901A870B07023FF03C08F81D9
:101B900081608F83B9016470707022FF03C08F81F0
:101BA00082608F83042F10E0C8018F7090700897B7
:101BB00009F04BC08F2D82958F70EAEAF2E0E80FB2
:101BC000F11DE491ED838D2D8095482F4F704830A5
:101BD00008F04051842F90E0880F991F880F991FBB
:101BE000909581959F4F8A838D2D90E0809590955B
:101BF000807F907095958795959587959595879514
:101C000095958795482F883008F04051842F90E0B3
:101C1000880F991F880F991F909581959F4F8983F1
:101C2000AB2B19F08F8181608F83672B19F08F8127
:101C300082608F8321FF03C08E8182608E8320FFAC
:101C400093C08E8181608E838FC0ED2CFF24C701ED
:101C5000807C9070803C9105D9F58FEFD81621F0EB
:101C600081E080937F010FC080917F01882359F428
:101C700021FF03C08E8182608E8320FF75C08E811C
:101C800081608E8371C020FF02C08FE78C8321FFAB
:101C900002C080E88B83E0FE02C08FE78B83E1FE09
:101CA00002C080E88C83E2FE03C08E8180648E8354
:101CB000E3FE03C08E8180688E83E4FE03C08E81C4
:101CC00082608E83E5FE50C08E8181608E834CC021
:101CD000C701807F9070009709F510927F0121FF66
:101CE00003C08E8180618E8320FF03C08E8182605D
:101CF0008E83E0FE03C08E8181608E83E1FE03C08F
:101D00008E8188608E83E2FE03C08E8180648E8324
:101D1000E3FE2AC08E8180688E8326C080389105BC
:101D200009F582E080938601842F0E94330D8F771E
:101D300000FD8195F50183830E945D0D182F0E949F
:101D4000330D8F7710FD8195F5018283E1FE03C08D
:101D5000818181608183E0FE07C0F501818182601D
:101D6000818302C010927F01DF91CF911F910F916B
:101D7000FF90EF90DF90BF90AF900895382F8FE0E5
:101D80008A95F1F790E020E0E5E2F0E04EE6A3E28C
:101D9000B0E030FF04C080818061808303C0808117
:101DA0008F7E808380818B7F8083842F8A95F1F75B
:101DB00026958C9185FD2068808184608083842FA6
:101DC0008A95F1F79F5F983011F03695E2CF8FE05A
:101DD0008A95F1F7822F0895CF92DF92FF920F93A9
:101DE0001F93CF93DF93EC016B01E4E2F0E080817D
:101DF0008D7D808380818C618083E5E2F0E080814D
:101E00008E6380838081877F80838FE08A95F1F75E
:101E100081E00E94BE0E82E40E94BE0E082F10E0F8
:101E2000813409F411E0FF24033711F4FF24F39403
:101E3000812F8F2990E020E030E0033511F421E07C
:101E400030E0822B932B892B09F484C08FEF0E9402
:101E5000BE0E8A3509F07EC08FEF0E94BE0EE82FBD
:101E6000982F80FD03C08F8182608F8393FD03C014
:101E70008F8181608F83112389F094FD02C080E8F7
:101E80008A8396FD02C08FE78A83EE2314F080E8F0
:101E9000898395FD1AC08FE7898317C0FF20A9F0B9
:101EA00091FD03C08F8184608F8392FD03C08F8179
:101EB00088608F83E295EF70F0E0E095F095EF7029
:101EC000F070E953FD4FE491ED838FEF0E94BE0E59
:101ED000282F982F80FD03C08E8180618E8391FD15
:101EE00003C08E8180628E8392FD03C08E818064E8
:101EF0008E8393FD03C08E8180688E8394FD03C022
:101F00008E8181608E8395FD03C08E8182608E8379
:101F100096FD03C08E8184608E8322231CF08E8107
:101F200088608E83FF2011F40335A1F48FEF0E94A7
:101F3000BE0E80588B838FEF0E94BE0E80588C831C
:101F40008FEF0E94BE0E805889838FEF0E94BE0ED5
:101F500080588A83033209F053C083E0809386015E
:101F60008FEF0E94BE0E8A3509F04AC08FEF0E94A3
:101F7000BE0EE82F83FD07C0D60115968C911597EC
:101F8000816015968C93E295EF70F0E0E095F09506
:101F9000EF70F070E953FD4FE491D6011396EC9386
:101FA0008FEF0E94BE0E282F83FD04C0F6018481AE
:101FB0008068848324FD07C0D60114968C91149701
:101FC000816014968C9325FD04C0F60184818260A3
:101FD00084838FEF0E94BE0E8058D60111968C9399
:101FE0008FEF0E94BE0EF60186838FEF0E94BE0E19
:101FF000D60117968C938FEF0E94BE0EF601808754
:10200000E5E2F0E08081886080838FE08A95F1F7D7
:10201000DF91CF911F910F91FF90DF90CF900895A6
:1020200090E0E3E2F0E003C09F5F983C19F080810C
:1020300081FDFACF089590E0E3E2F0E003C09F5FF6
:10204000983C19F0808181FFFACF08950F931F9378
:10205000CF93DF93EC01E4E2F0E080818D7C80831C
:1020600080818C608083E5E2F0E080818E638083F4
:10207000EAE2F0E080818E7E8083EBE2F0E0808116
:10208000816180838AE08A95F1F7489B57C04C991B
:1020900003C08E8180648E83E5E2F0E08081877FDB
:1020A00080838AE08A95F1F71C9902C080E88A83D0
:1020B0001D9902C08FE78A83489902C080E889830E
:1020C0004C9902C08FE78983E5E2F0E08081837F4D
:1020D000886080838AE08A95F1F71C9903C08E811D
:1020E00082608E831D9903C08E8184608E8348999F
:1020F00003C08E8181608E834C9903C08F81816083
:102100008F83E5E2F0E08081837F80838AE08A9597
:10211000F1F71C9903C08E8180628E831D9903C0E4
:102120008E8180618E83489903C08E8188608E8302
:102130004C993AC18E8180688E8336C11C9B34C114
:10214000E5E2F0E08081877F808380818B7F8083E0
:102150000E9410101C990EC105E210E0F801808168
:10216000846080830E941B10F80180818B7F8083B4
:102170000E9410101C9902C080E88A831D9902C039
:102180008FE78A83489902C080E889834C9B02C00C
:1021900010E010C08FE7898310E00CC09260489B6C
:1021A00094604C9B9860EAEAF2E0E90FF11DE4913B
:1021B000ED8311E0E5E2F0E08081846080830E949D
:1021C0001B101C9903C08E8182608E831D9903C0F1
:1021D0008E8184608E83489903C08E8181608E8356
:1021E0004C9903C08F8188608F83E5E2F0E08081A5
:1021F0008B7F80830E9410101C9903C08E818062A7
:102200008E831D9903C08E8180618E83489903C09F
:102210008E8188608E834C9903C08E8180688E8306
:10222000E5E2F0E08081846080830E941B104C997D
:1022300003C08E8180648E83E5E2F0E080818B7F35
:1022400080830E9410101C9902C000E101C000E0D0
:102250001D9B0062489B00644C9B0068E5E2F0E037
:102260008081846080830E941B101C9B01601D9BE9
:102270000260489B04604C9B0860113019F48FE7A2
:10228000801B8983E5E2F0E080818B7F80830E9460
:1022900010101C9902C000E101C000E01D9B00620B
:1022A000489B00644C9B0068E5E2F0E0808184601C
:1022B00080830E941B101C9B01601D9B0260489B39
:1022C00004604C9B0860113019F48FE7801B8A83EF
:1022D000E5E2F0E080818B7F80830E9410101C99E2
:1022E00002C000E101C000E01D9B0062489B006449
:1022F0004C9B0068E5E2F0E08081846080830E946E
:102300001B101C9B01601D9B0260489B04604C9B42
:102310000860113019F4802F80588C83E5E2F0E0DA
:1023200080818B7F80830E9410101C9902C000E185
:1023300001C000E01D9B0062489B00644C9B00684C
:10234000E5E2F0E08081846080830E941B101C9B8A
:1023500001601D9B0260489B04604C9B086011302B
:1023600019F4802F80588B83E5E2F0E080818C6047
:1023700080831AC005E210E0F801808184608083C8
:102380000E941B10F80180818B7F80830E941010B7
:10239000E3E2F0E0808182958F708095982F9170B4
:1023A000808185FFFBCEFBCEDF91CF911F910F91F6
:1023B0000895DC01E4E2F0E08081817C8083E5E245
:1023C000F0E080818E638083E7E2F0E08081827CB0
:1023D0008083808182608083E8E2F0E080818F6387
:1023E000808380818D7F808380818260808390E87C
:1023F0002FE0E3E2F0E0822F8A95F1F7808185FFFC
:1024000003C011969C931197808184FF03C012969C
:102410009C931297808183FF03C013969C9313971C
:10242000808182FF03C014969C9314979F5F9F370F
:1024300011F711968C9111978E3719F411961C9201
:10244000119712968C9112978E3719F412961C924E
:10245000129713968C9113978E3719F413961C923A
:10246000139714968C9114978E3719F414961C9226
:102470001497309907C016968C911697816016961E
:102480008C931697199907C016968C9116978260AF
:1024900016968C9316974C9907C016968C911697A2
:1024A000846016968C931697489906C016968C9160
:1024B0001697886016968C930895E9E6F0E080817F
:1024C00082608083EDE3F0E0808181608083E4EAD4
:1024D000F1E08BE4808331978AE5808308951F9330
:1024E000CF93DF938091B401982F93500AF4B4C036
:1024F0002091B1018091B0018D3209F0ABC09830CC
:1025000009F0A8C08CE090E0821B9109FC01E8541E
:10251000FE4FEF0183EC809398018AE580932201BE
:10252000109280018081807629F0CF010E945704AB
:10253000282F87C092811092A1018181882331F4D4
:10254000E2EAF1E0108222E0319777C0853031F481
:102550009093B50120E0E1EAF1E06FC0863009F028
:102560004CC08381813031F4CF010E947D04282F3B
:1025700080E440C0823031F4CF010E947D04282FD6
:1025800080E038C0833009F5992349F484ED92E066
:102590009093B3018093B20180E424E02BC091308A
:1025A00049F488ED92E09093B3018093B20180E406
:1025B0002AE020C09230E1F482EE92E09093B301E1
:1025C0008093B20180E42CE115C0813249F482E1AC
:1025D00091E09093B3018093B20180E429E00AC0B6
:1025E000823231F4CF010E947D04282F80E402C0A2
:1025F00080E420E08093800124C0883021F421E031
:10260000E7EBF1E01AC0893031F49093B70120E094
:10261000E1EAF1E012C08A3021F421E0E1EAF1E0E0
:102620000CC08B3021F020E0E1EAF1E006C08BE441
:102630008093A40120E0E1EAF1E0F093B301E0939C
:10264000B2018F81882321F48E81821708F4282F0C
:10265000209323011092B4018091220184FF57C07E
:10266000109123011F3F09F452C0193008F05CC0DB
:1026700010922301E8E9F1E0808198E889278083BE
:10268000112309F45DC02091B2013091B301809112
:10269000800186FF14C0A9E9B1E080E090E0F90173
:1026A000E80FF91FE491ED9301961817C1F7812FF8
:1026B000815090E00196F901E80FF91F0FC0D90190
:1026C000912FE9E9F1E08D9181939150E1F7812F0C
:1026D000815090E00196F901E80FF91FF093B301E2
:1026E000E093B201193068F489E991E0612F0E940A
:1026F000EA13612F6C5F6C3040F48FEF80932301FD
:1027000004C08FEF809323016EE16093220194E176
:10271000E9E2F0E080818670D1F49150D9F710920F
:10272000B5011092AF0113C0812F8850809323010F
:10273000E8E9F1E0808198E88927808318E0A3CF59
:1027400089E991E060E00E94EA1364E0D6CFDF916E
:10275000CF911F910895FF920F931F93DC01F62EE6
:102760008091A30184FF07C0E4EAF1E0808198E84A
:102770008927808303C08AE58093A3019F2DE5EA22
:10278000F1E08D9181939150E1F705EA11E0C801E4
:102790006F2D0E94EA138F2D8C5F02501040F801BC
:1027A00080831F910F91FF900895A82FB92F80E08B
:1027B00090E041E050EA609530E009C02D91822719
:1027C0009795879510F084279527305EC8F36F5F43
:1027D000A8F30895EADF8D939D930895CF93CFB723
:1027E000CF93C395499BE9F7499B0BC0499B09C00F
:1027F000499B07C0499B05C0499B03C0499B01C039
:10280000C2C0C091B101DF93DD27C854DE4F2F93C2
:102810002FEF499B03C02F91DF91E6CF0F931F93BA
:102820004F936F9309B101FB20F93F933BE05F9316
:102830001EC04E7F012F19B11670E1F0216000001B
:102840001DC0102F4D7F2260000009B1067091F06D
:102850001DC04B7F2460012F000019B1167051F08C
:102860001EC019B1167031F0477F28601BC019B126
:10287000167009F462C04FEF297FD9F2012701FBDE
:1028800021F909B10670B1F3237FD9F2102711FBAA
:1028900022F900C019B1167069F3277ED1F2012721
:1028A00001FB23F92F7CE9F209B1067019F3102717
:1028B00011FB24F92F7929F100C019B11670E9F143
:1028C000012701FB25F92F7311F100C009B1067032
:1028D000A1F1102711FB26F92230F8F000C019B140
:1028E000167059F1012701FB27F92430E0F0422747
:1028F000000009B14993102711FB20F93150C8F0AD
:10290000B6CF4F7E09B10670C1F02061D3CF2062EF
:1029100019B1167091F04F7DD6CF4F7B09B106707B
:1029200061F02064D9CF4F7719B1167031F020686B
:10293000DCCF11E01CBB002719C03B503195C31BF5
:10294000D04011E01CBB0881033C09F10B34F9F0C5
:102950002091AF011981110F1213EDCF4A81441F4D
:10296000093651F10D3211F0013E29F70093B601FD
:102970005F913F916F914F911F910F912F91DF9137
:10298000CCB3C0FD2ECFCF91CFBFCF911895209162
:10299000B601222369F31091B401112389F5343073
:1029A0008AF13093B4012093B0011091B1013BE062
:1029B000311B3093B10126C00091B401013004F500
:1029C0000AE54F7049F43091220134FD1CC0009398
:1029D0002201C8E9D1E01BC03091A30134FD13C02E
:1029E0000093A301C4EAD1E012C00527112700001B
:1029F00019C0052711271FC005271127000024C073
:102A00004AE502C032ED432FC4E1D0E032E01AB112
:102A10001660599A0BB11AB956E020E866E020FF1B
:102A2000052727950BB917951C3FF8F66A95B9F756
:102A300020FF0527279500000BB917951C3FC8F606
:102A400020FF05272795179566E01C3F0BB9A0F6D8
:102A500029913A9521F7097F1091B501110F0BB912
:102A6000C651D04011F01093AF0111E01CBB0260C1
:102A70001AB1197F402F497F53E05A95F1F700C0F2
:0C2A80000BB91AB94BB974CFF894FFCF12
:102A8C000902220001010080FA0904000001030080
:102A9C0000000921010100012250000705810308F3
:042AAC0000085AFFC5
:00000001FF
